:100000000C940D030C943D030C943D030C943D03A0
:100010000C943D030C943D030C943D030C943D0360
:100020000C943D030C943D030C943D030C943D0350
:100030000C943D030C943D030C943D030C943D0340
:100040000C943D030C943D030C943D030C943D0330
:100050000C943D030C9417050C943D030C943D0344
:100060000C943D030C943D030C943D030C943D0310
:100070000C943D030C943D030C943D030C943D0300
:100080000C943D030C943D030C943D030C943D03F0
:100090000C943D030C943D030C943D030C943D03E0
:1000A0000C943D030C943D030C943D030C943D03D0
:1000B0000C943D030C943D030C943D030C943D03C0
:1000C0000C943D030C943D030C943D030C943D03B0
:1000D0000C943D030C943D030C943D030C943D03A0
:1000E0000C943D030C94660302F6FFF40102F7FF43
:1000F000F40102F8FFF40102F9FFF40102FAFFF43F
:100100000102FBFFF40102FEFFF40102FEFFF40115
:1001100002FEFFF4010000000000300C03DF31FAA2
:100120002B78D5D86C2945A1026969918D6571B884
:1001300043DEF2F6786E1DBF344ECB382EFD3259B9
:10014000750732E231778433E1EDC56E523627967A
:1001500015198D8D88AB4DBCF918F5271627818CA4
:100160002FB46E602BF2940CE0597B338FA3C9A49B
:10017000BD573245027F02FB98F723AE1EA53A4DCC
:1001800059A9AE849B42917C9B0CB02BB07ACF6D69
:10019000D102B2D381B4CE19ACF2C7CB970218F01A
:1001A000ABC774470906C4A51374D0C3EEA030BF13
:1001B000A2E2922497613D4453050FEA0728DAB37F
:1001C000EF4FFAF955BE9F68336F2B21105CE0B2F8
:1001D0003F73D6D7D4141B271A2A122153ECD542C9
:1001E0003CCF3C918EDBFAC24B26E35B82C40EC14E
:1001F00037E5980BFAB43314DE453631320B746EA2
:10020000DBB1006A8CFA2CD7210F33A3D342650AE5
:1002100027FE1621B24935918E6BC3C077382E5216
:10022000E92FBC7629E84D4BF781EFCBC354D5EBD2
:1002300053EC0D06354398C3AF5B842694B3787DA9
:10024000E235F30C1D415715C346E0879BB672EEAD
:10025000A37FF5D8C28D9C72E920987DD311FBB5A0
:1002600046EFC164311979F45F5A7BFA11EEE9B4B3
:100270006EDE8C316C29A355493BD31C4DCED293F5
:10028000BE94F7EFAD71E40DCC6008DD4EF192BC89
:10029000D01FED3C48909291CC65AE193481ADF2FF
:1002A00015A5E2C317C6D0E327D8C175CA53329B40
:1002B000721FD8BBB06A4D7DD0FB97047D45F79384
:1002C000EAD95601A027E4C700A53DCBF96F666CBB
:1002D0008F3F2740A974BE7A70557FEE9A7681854C
:1002E00050D787F1FF6BB9FF11F7CA0B673177F76A
:1002F000709F371A14F694854B1373E68AF46CDBFF
:10030000CBF3CCCB5F86CA717D957CE4C6F4DC363A
:10031000931350A70AE52D55F9A03C8394A95F607B
:100320009C2B2BFCB2F66D308BE91451DEF08871FA
:1003300004D8190EBE4664B7E6A13B7B4A9ADBE7B8
:10034000C607E378FD51A8883BBDDA19AE628AB3CF
:100350003AA4C2F9EB26B0D2C8EC4D138629FA4D67
:1003600030DEC62E2F6FB66A2D9083DBF20E8F2DF6
:10037000B351279E78D87140C4BE544BE84E9818AC
:100380002D5F465DCEFDC7FB8E4BD7815A66AF0E03
:10039000B7D6AC2FAE1D7072DCC4BDC41356DD40A1
:1003A000B6249D84216580B0B157310BBDE019752D
:1003B000B6C6A564E415D7C1DA9585EDEC632EA227
:1003C00087CC26A932A659E3FD8AEFBB6B09302101
:1003D000CFD586B4EB5D75C5F3FBB3DF5EE281E696
:1003E000AFA78FE14EE8C54C73B407DFBE38018E6E
:1003F0000D8742F8E5B8BED8B472B7125439F90483
:10040000E088E62F71AB7BE56083C41EBBC5ACC939
:100410004DEFC233A7800C5BF3C36E48FC674CDD25
:10042000F0320D61DD88473E0B0B5CC7D109901E91
:10043000F852529FD25EFBC622690E1FD15AFDC2EE
:100440008C0A236A926AA99E760565470EF56606B0
:1004500047B9A61A17A2E0390CEE59DD49569FD6C6
:1004600060C341F32EEA91A4F0F7ECFEEC5305349F
:100470000CAC4F244E2F5D5A1EB738670DD83E6D19
:100480009C7F61CA69F26F59E95C58D6B05E0BBCBB
:100490000A5AE0598A3EB4A8F5EC1003C54E7161C2
:1004A000CED22C37C49C91AEF8EA85A8489065520C
:1004B000EB46AC7584601E7A4D2F7D137DEE744C37
:1004C000C0A183853D153436FFBADF474B449A36C9
:1004D0008A47AC0FA7CA89F5F9070877F57DC3B637
:1004E0001F473C5C5C71935C2B72A376B73EAC41BA
:1004F0008558512D23DB221CE22B93D8A8578FC798
:100500009ECB24FB3CB757682AFBDEE1398B23BF27
:10051000E474EC074F0F24323AB87F8285888C8FC1
:100520009295989B9EA1A4A7AAADB0B3B6B9BBBE45
:10053000C1C3C6C9CBCED0D3D5D7D9DCDEE0E2E487
:10054000E6E8E9EBEDEEF0F1F2F4F5F6F7F8F9FA9A
:10055000FBFCFCFDFDFEFEFEFEFEFEFEFEFEFEFDC5
:10056000FDFCFCFBFAFAF9F8F7F6F4F3F2F0EFED24
:10057000ECEAE8E7E5E3E1DFDDDBD8D6D4D1CFCCA8
:10058000CAC7C5C2BFBDBAB7B4B1AFACA9A6A3A014
:100590009D9A9693908D8A8784817D7A7774716E07
:1005A0006B6864615E5B5855524F4D4A4744413F0A
:1005B0003C393734322F2D2A282623211F1D1B19A1
:1005C00017161412110F0E0C0B0A08070605040467
:1005D0000302020101000000000000000000000111
:1005E000010202030405060708090A0C0D0E10118A
:1005F000131516181A1C1E20222527292B2E3033DE
:1006000035383B3D404345484B4E5154575A5D6049
:100610006366696C6F7276797C7F11241FBECFEFA1
:10062000D1E2DEBFCDBF00E00CBF84B780930D04E4
:1006300014BE0FB6F894A8958091600088618093ED
:100640006000109260000FBE13E0A0E0B2E0ECE0AA
:10065000FCE000E00BBF02C007900D92AA3FB1077B
:10066000D9F724E0AAEFB3E001C01D92AD30B20784
:10067000E1F70E94BC050C9404060C940000CF9393
:10068000C62F0E943F058FEF80BBC1BBEBE0F1E0BE
:100690008081857F808385E08A95F1F700008081E5
:1006A0008A608083CF9108950E943F0510BA11BAE5
:1006B000EBE0F1E08081837F808385E08A95F1F72C
:1006C00000008FB190819C6090830895CF92DF925B
:1006D000EF92FF92CF93C82F80E4C82E82E4D82EE9
:1006E0008FE0E82EF12C85E00E94540385FD06C0C2
:1006F00081E0C81AD108E108F108A9F76C2F80E061
:100700000E943F0390E080E0CF91FF90EF90DF9058
:10071000CF90089563E883E00E943F0363E080E0A8
:100720000E943F0360E081E00E943F0363E083E0BA
:100730000E943F0380E092E090930A0480930904B2
:100740008CE592E00C94D805CF93C62F0E943F050C
:100750008FEF80BBC1BBEBE0F1E080818D7E8083B9
:1007600085E08A95F1F70000808180618083808137
:1007700082608083CF9108950E943F0510BA11BA1C
:10078000EBE0F1E080818B7E808385E08A95F1F754
:1007900000008FB190819461908308950F931F930F
:1007A000CF93DF9380910F02833009F4B3C0A8F494
:1007B000813009F444C0CFE7823009F476C0C0E04C
:1007C00060E08C2F81700E94A403CF5FCF3FC1F700
:1007D000DF91CF911F910F910895843009F4C8C023
:1007E0001FE7CFEFD0E00FEF853049F760910004AD
:1007F0008FEF860F8E3F28F080910E0281958093B7
:100800000E0280E00E94A4036091000481E00E9437
:10081000A4034091FA035091FB0357FDDFC0809180
:10082000FE039091FF030196841795070CF0CAC050
:100830009093FF038093FE031150C1F6C9CFCFE719
:10084000E0910004F0E0E65EFA4F649181E00E94DE
:10085000A403E0910004F0E0E65EFA4F649180E0CA
:100860000E94A4032091FA033091FB0337FD19C0C5
:100870008091FE039091FF030196821793073CF449
:100880009093FF038093FE03C150D1F6A1CF109245
:10089000FF031092FE03809100048F5F8093000499
:1008A000F3CF80910004821BF9CF8091000487FF71
:1008B0001DC06FEF80E00E94A4036FEF81E00E94F3
:1008C000A4032091FA033091FB0337FD1FC08091F0
:1008D000FE039091FF030196821793076CF49093A7
:1008E000FF038093FE03C15001F772CF60E080E008
:1008F0000E94A40360E0E2CF1092FF031092FE0377
:10090000809100048F5F80930004EDCF80910004FC
:10091000821BF9CFCFE76091000480E00E94A4031E
:100920006091000481E00E94A4032091FA033091B9
:10093000FB0337FD19C08091FE039091FF030196E0
:10094000821793073CF49093FF038093FE03C150FA
:1009500011F73ECF1092FF031092FE038091000426
:100960008F5F80930004F3CF80910004821BF9CF46
:10097000CFE7E091FC03F091FD03E65EFE4F64914A
:1009800081E00E94A403E091FC03F091FD03E65E88
:10099000FE4F649180E00E94A4038091FC0390913B
:1009A000FD030196811524E0920738F49093FD032E
:1009B0008093FC03C150E9F60BCF1092FD03109217
:1009C000FC03F8CF1092FF031092FE038091000405
:1009D00090910E02890F809300042ECF20910E0279
:1009E0002403B001259F700D112480910004FE01A5
:1009F000E81BF109E617F7071CF4009300041CCF6D
:100A0000249F202D11242093000416CF80E00E9403
:100A1000BC0380FF0C94CE03089582E884BD84E07B
:100A200085BD80E487BD82E080936E0008951F92AB
:100A30000F920FB60F9211240BB60F922F933F9384
:100A40004F935F936F937F938F939F93AF93BF93D6
:100A5000EF93FF930E946C05FF91EF91BF91AF91CF
:100A60009F918F917F916F915F914F913F912F91C6
:100A70000F900BBE0F900FBE0F901F901895809394
:100A8000080108958FEF80BB8093070180930A01CE
:100A90001092080111BAEBE0F1E0108280818F61C1
:100AA00080838FE891E00197F1F700C0000080811A
:100AB0008E7F8083089585E00E94540380FF07C0E5
:100AC00080E00E945403682F80E00E943F030E9450
:100AD000060590E080E00895609105047091060499
:100AE0006F5F7F4F7093060460930504E0910104EB
:100AF000F09102048081918140910304509104049B
:100B0000E5E0E49F9001E59F300D1124FC01E20F28
:100B1000F31F3396A591B4916A177B0738F54F5FA1
:100B20005F4FFC01E20FF31F389625913491232B80
:100B3000F1F0509304044093030420910304309196
:100B4000040445E0429FF001439FF00D11248E0FF5
:100B50009F1FFC012591349120930F020196FC0107
:100B6000859194919093FB038093FA0308951092DA
:100B7000040410920304E1CFF8940E9442050E94FD
:100B80008A030E940D0588EE90E090930204809302
:100B90000104789488E19EE00FB6F894A8958093BC
:100BA00060000FBE90936000A8950E945B05FCCF8B
:100BB0000F931F93CF93DF93E0910904F0910A0400
:100BC000238110E000E021FD0EC00FEF1FEFC801F0
:100BD000DF91CF911F910F9108951995892B11F0F5
:100BE0000FEF1FEFCE01EC01899160910904709124
:100BF0000A04DB011896ED91FC918111EECF8AE099
:0C0C00001995892B21F3E1CFF894FFCF68
:100C0C00000000020000000066030000000001016B
:100C1C0062026E027B027F02870294029D02A40292
:100C2C00B702C502CF02DA02E402F002F602FF02BA
:100C3C000D03130319031E03230329032D0333038D
:100C4C0046035A0374037B03810387038C039103CC
:100C5C00A203AA03B603CC03DB03EA03494E4954AF
:100C6C000D00464C4F505059204449534B005343B0
:100C7C0052455720445249564552004B4559005352
:100C8C0041555341474500524F5454454E20464C14
:100C9C00455348004B4559424F415244005049532B
:100CAC00544F4C004E4F5448494E474C4F4E454CB8
:100CBC005920524F414400532F4E20444952542046
:100CCC00524F41440046495245504C414345004E19
:100CDC002F5720537472656574004F4C4420484F55
:100CEC00555345004C4956494E4720524F4F4D00E5
:100CFC00415454494300424153454D454E540043E1
:100D0C004F4D505554455220524F4F4D006E6F72FF
:100D1C00746800736F75746800776573740065612F
:100D2C0073740073686F6F7400757365004552526D
:100D3C004F5200596F752063616E277420646F20C9
:100D4C00746861742100596F752063616E2774207B
:100D5C007573652074686174210057686174206133
:100D6C00726520796F7520676F696E6720746F20CC
:100D7C00646F3F00676F696E6720004E4F52544896
:100D8C0000534F5554480045415354005745535454
:100D9C0000594F55204D415920414354204E4F5737
:100DAC00210069742064696564006974207375722C
:100DBC0076697665640061206265617220626C6F91
:100DCC00636B732074686520776179006974207295
:100DDC00616E20617761792E2E2E00697420776FF9
:100DEC006E277420737461727400796F752063615F
:0A0DFC006E27742074797065000002
:00000001FF
